:020000040000FA
:060000004DEF0BF01200B1
:060800004DEF0BF01200A9
:06082A000100B2160000FF
:08083000FD00000003000000C0
:08083800040120511F0B01080F
:1008400001E012002051600BE842E842E842E84231
:10085000E842010801E01200245103E0240501E010
:1008600012002151230A43E0010A3BE0030A2BE076
:10087000010A20E0240A3BE0070A39E0010A37E0D8
:10088000030A10E0010A01E012000101030E0B6FE0
:100890000101F50E0C6F000E0D6F010113930101A4
:1008A000080E1DD00101030E0B6F0101F50E0E6F36
:1008B000000E07D00101030E0B6F0101EA0E0E6F4F
:1008C000000E0F6F12000101030E0B6F0101EA0E03
:1008D0000C6F000E0D6F010113930101070E106FD5
:1008E00012000101030E0B6F22C4F1F0120012007E
:1008F0000001EA6BC20EEB6F010EEC6FED6BEE6B5D
:10090000EF6B080EF06FE36BE26B1A0E726E1E0E49
:10091000736E0401000E166F050E176F400E146FF4
:100920000401196F080E1A6F050E1B6F880E186FE1
:100930000401480E1E6F050E1F6F400E1C6F120043
:10094000D9CFE6FFE1CFD9FF0001E26B040118BF68
:1009500030D0FC0EDBCF02F01951D880025403E2F4
:10096000FC0E19C4DBFF0001E26BFC0EDB50E25D04
:1009700019E2E251EA6A080FE96E050EEA22EF5029
:10098000E66EE251E76EFD0EDBCFE9FFFE0EDBCF38
:10099000EAFFE750E926000EEA22E552E750EF6E43
:1009A000E22BE3D70401400E196F1817187D880E4B
:1009B00018130001E251E552E7CFD9FF1200D9CF59
:1009C000E6FFE1CFD9FFE6520001E3512EE1DF6AF5
:1009D000DF2ADF50026E036AFF0E021802E10350A5
:1009E0000BE0FD0EDBCFE9FFDB2AFE0EDBCFEAFFDB
:1009F00001E3DB2AEF50ECE1DF50026E036AD950CD
:100A0000FD0FE96EFF0EDA20EA6E0250EE5E035033
:100A1000ED5AFD0EDBCFE4F0FE0EDBCFE5F0DFCFCD
:100A2000E8F00001E96B010EE36FE552E552E7CF14
:100A3000D9FF1200D9CFE6FFE1CFD9FFE65200017E
:100A4000E3512FE1DF6ADF2ADF50026E036AFF0EF7
:100A5000021802E103500CE0FD0EDBCFF6FFDB2AAB
:100A6000FE0EDBCFF7FF01E3DB2A0800F550EBE1D8
:100A7000DF50026E036AD950FD0FE96EFF0EDA20D7
:100A8000EA6E0250EE5E0350ED5AFD0EDBCFE4F04D
:100A9000FE0EDBCFE5F0DFCFE8F00001010EE96FDD
:100AA000E36FE552E552E7CFD9FF1200D9CFE6FF59
:100AB000E1CFD9FFE65204011CBF66D0030E00014E
:100AC000E35D01E1E36BE3515FE0020EE35D03E10F
:100AD00004011D6B50D0E30551E1400E026E036A24
:100AE000E851025C000E035803E2400EDF6E02D0B4
:100AF000E8C0DFFFDFCF1DF4DF50E85DE86F480E90
:100B0000E66F050EE76FE90514E1DF5025E0E4C06C
:100B1000F6FFE5C0F7FF0800F550E6C0E9FFE7C0C3
:100B2000EAFFEF6EE62B000EE723E42BE523DF065A
:100B3000ECD7DF5011E0E4C0E9FFE5C0EAFFEF5079
:100B4000E6C0E9FFE7C0EAFFEF6EE62B000EE72301
:100B5000E42BE523DF06EDD70001E8510FE10401A6
:100B60001D51026E036A400E021805E1035003E1B5
:100B70000001020E02D00001030EE36F400E0401DB
:100B80001C171C7D880E1C13E552E552E7CFD9FFD8
:020B9000120051
:0E0B92006C5002E0000E01D0010E00090BE0D5
:100BA000040100513C0BE842E8420D0802E1E4EF89
:100BB00005F019EF06F06C5002E0000E01D0010EB6
:100BC000040901E045D81200D9CFE6FFE1CFD9FFF3
:100BD000E65201010A6B0B6B106B116B44EC07F0D2
:100BE000DF6ADF50026E036A010E025C000E0358DA
:100BF0001AE201010B5117E1F76ADF34FE0BF736F9
:100C0000F66EA50EF626150EF7220900F5CF02F0B6
:100C10000800F5CF03F004D003C0FAFF0250F96ECC
:100C2000FBDFDF2ADED7DDD8E552E552E7CFD9FF7B
:100C30001200020E01010A5D09E194D8040100BD11
:100C400002D0C80E01D0880E006F120036EF07F0F8
:100C5000040E0101125D09E122C46EFF6E5000080E
:100C600002E2050E01D0030E126F01010A0509E12F
:100C70000AD8040104BD02D0C80E01D0880E046F4A
:100C8000120036EF07F0D9CFE6FFE1CFD9FF020E11
:100C9000E1260101080E105D000E115905E210C198
:100CA000DEFF11C1DDFF03D0080EDE6EDD6A040138
:100CB00004930491010EDB500413DFCF05F4000E02
:100CC000DB500101105F010EDB50115B280E0E6F2F
:100CD000040E0F6F010113A31DD0D9CFE9FFDACFA6
:100CE000EAFFEE50ED1032E00CC1F6FF0DC1F7FF48
:100CF0000800F5500EC1E9FF0FC1EAFFEF6E0101D8
:100D00000E2B000E0F230C2B0D23DF06010EE5E248
:100D1000DB06E3D7D9CFE9FFDACFEAFFEE50ED10DB
:100D200015E00CC1E9FF0DC1EAFFEF500EC1E9FF6C
:100D30000FC1EAFFEF6E01010E2B000E0F230C2BEB
:100D40000D23DF06010EE6E2DB06E4D7F56E020EA8
:100D5000E15C02E2E16AE552E16EF550E552E7CF6F
:100D6000D9FF1200D9CFE6FFE1CFD9FF020EE1266D
:100D7000030E04010015E76E010EE7CFDBFF01C48F
:100D8000DFFFDE5001011027DD501123280E0C6F0C
:100D9000040E0D6FD9CFE9FFDACFEAFFEE50ED1068
:100DA00014E00CC1E9FF0DC1EAFFEF500EC1E9FFED
:100DB0000FC1EAFFEF6E0E2B000E0F230C2B0D233D
:100DC000DF06010EE7E2DB06E5D7F56E020EE15C19
:100DD00002E2E16AE552E16EF550E552E7CFD9FF54
:100DE000120001010B510BE10401080E016F200EEE
:100DF000026F040E036F840E006F040123D0040100
:100E000020AF22D0010110510401265D01011151D2
:100E10000401275904E226C410F127C411F133DF7D
:100E20000101010E0A6F0401080E016F200E026F0E
:100E3000040E036F800E006F0401280E066F040E6F
:100E4000076FC80E046F10D00101020E0A6F040173
:100E5000056BC80E046F0401080E016F280E026FA7
:100E6000040E036FC80E006F6D98120001010A6B2B
:100E70000401080E016F200E026F040E036F880E2E
:080E8000006F0401046B120075
:080E880004012051600BE84257
:100E9000E842E842E842E842000901E0120021513C
:100EA000070A4CE00B0A4AE0070A3BE0010A27E088
:100EB0000B0A23E0020A21E0030A1DE0080A12E0FF
:100EC000010A0EE00F0A0AE0030A01E01200010124
:100ED000010E0B6F0101040E126F12009FEF07F05D
:100EE000F6EF07F00101010E0B6F0101140E0C6FFC
:100EF000010E0D6F10D01DEF08F068EF08F0010132
:100F0000010E0B6F0401245101010C6F0D6B150EC6
:100F10000C27010E0D23010113930101010E106F27
:100F200012000101010E0B6F04012451EA6A150F32
:100F3000E96E010EEA2222C4EFFF12001200800EB9
:100F40000401205D52E12351030A30E0010A0CE064
:100F5000030A49E10101010E0B6F0101E60E0C6F5E
:100F6000140E0D6F120E3CD00101010E0B6F040127
:100F70002251F66EF76AD890F636F7369B0EF626B3
:100F8000150EF7220900F5CF0CF10A00F5CF0DF18F
:100F9000020E0101F76A0C25F66E0D51F7220900C9
:100FA000F5CF10F10A00F5CF11F11DD00101010EAE
:100FB0000B6F04012251F66EF76AD890F636F736B9
:100FC0009F0EF626150EF7220900F5CF0CF10A0048
:100FD000F5CF0DF10CC1F6FF0DC1F7FF0800F5507C
:100FE0000101106F116B0101138312000101010E49
:100FF0000B6F0F0EE66E710EE66E0F0EE66E5EEC78
:101000000AF0E552E552E552010EE66E150EE66E67
:10101000010EE66E5EEC0AF0E552E552E55222C49E
:1010200014F10401225104E10101050E126F1200B6
:101030000101060E126F78EF04F00401286B296B92
:10104000040120511F0B020A13E0030A0DE0010AFC
:1010500031E10101010E0B6F04012881010113A18F
:1010600029D00401288326D00101010E0B6F22D064
:101070000101010E0B6F040124510F0B080DF350F9
:10108000036A000F026E040E03222451800B01E05C
:10109000010E040DF350010102240E6F000E032017
:1010A0000F6F0EC1E9FFEA6EEF50040B03E004017D
:1010B000010E286F01010B050AE10101280E0C6FDA
:1010C000040E0D6F010113930101020E106F120047
:1010D0000401220510E120511F0B00090CE1010160
:1010E000010E0B6F030E0401215D03E10101138169
:1010F00002D001011391040122513AE120511F0B4A
:10110000020836E124510F0B000932E00101010E03
:101110000B6F040124510F0B080DF350036A000FED
:10112000026E040E03222451800B01E0010E040D17
:10113000F350010102240E6F000E03200F6F030E07
:101140000401215D07E1840E0EC1E9FF0FC1EAFF32
:10115000EF6E120024AF06D00EC1E9FF0FC1EAFF07
:10116000EF6A1200880E0EC1E9FF0FC1EAFFEF6EB1
:0211700012006B
:0E117200FC0E8B16941694848250040B01E040
:10118000010E0001606F896A92688A68936A120092
:10119000D9CFE6FFE1CFD9FF030EE126DF6A010ECA
:1011A000DB6A020EDB6AA9D8060E0101125D01E2BC
:1011B00098D06D50020B01E094D0200EE66E610EC7
:1011C000E66E000EE66EA0EC04F0E552E552E55244
:1011D000DF6EDFCF02F0000EE76E0218E8AE02D03D
:1011E000023403D0E750D880025401E37AD0020ED3
:1011F00061C0DBFFDBA007D0010EDB508009E76E8A
:10120000010EE7CFDBFF020EDBA207D0010EDB50A1
:101210004009E76E010EE7CFDBFF020EDBA407D02B
:10122000010EDB502009E76E010EE7CFDBFF020E57
:10123000DBA607D0010EDB501009E76E010EE7CFE9
:10124000DBFF020EDBA807D0010EDB500809E76EBA
:10125000010EE7CFDBFF020EDBAA07D0010EDB5049
:101260000409E76E010EE7CFDBFF020EDBAC07D00F
:10127000010EDB500209E76E010EE7CFDBFF020E25
:10128000DBAE07D0010EDB500109E76E010EE7CFA0
:10129000DBFF010EDB508A6E8B720001FD510EE008
:1012A0000001E3511EE10001FD6B780EE66E160EA3
:1012B000E66E1AEC05F0E552E55213D00001E35159
:1012C00010E180CFA1F00001A26B0001A10EE46F3C
:1012D000000EE56F0001010EE86F0001E96B0001EF
:1012E000E36FF56E030EE15C02E2E16AE552E16E46
:1012F000F550E552E7CFD9FF12000001FE51FF1172
:1013000004E1500EFE6FC30EFF6FFE07000EFF5B81
:101310006DA204D0FE51FF111BE103D00101125157
:1013200002E18B901200120509E0020E125D06E048
:10133000030E125D03E0050E125D02E18B801200C8
:10134000060E125D05E10001FE51FF1101E18B70F7
:1013500012008250040B01E0010E0001605D07E005
:101360008250040B01E0010E606F82A4010C000C9E
:101370006DA60CD80101120508E16DBA06D0686AA5
:10138000696A69806988020E126F12006D6A696A63
:101390006D860101010E126F12006D6A696A01010A
:1013A000126B1200CDEF09F00101125101E11200A0
:1013B0006850040B04E06950040B01E03CD86DB2A6
:1013C00012006850010B04E06950010B01E054D891
:1013D0006850100B04E06950100B01E024D86850ED
:1013E000400B04E06950400B01E03BD86850200BF3
:1013F00004E06950200B01E036D86850020B04E08D
:101400006950020B01E036D8030E0101125D01E2C2
:1014100012006850080B06E06950080B03E0C9ECA5
:1014200005F068961200698468986D82A19AA08A76
:101430000300A09A12006D92699468941200010151
:1014400013A10ED0F8DF6D840101080E166F070E90
:10145000176F1607000E175B16511711FAE16D94FE
:101460001200689C120070A003D036EC07F0709058
:10147000689A1200689212006A6A686A9F0E6B6E20
:101480007B0E696E6E6A0F0EE66E710EE66E0F0EC3
:10149000E66E14D8E552E552E552160E706E68A657
:1014A00002D06896FCD76D9836EC07F001011391D5
:1014B0000101146B0101030E126F1200D9CFE6FF78
:1014C000E1CFD9FFFD0EDBCFE9FFFE0EDBCFEAFF58
:1014D000FC0EDB5004E0EE6AFC0EDB06F9D7E552A9
:0614E000E7CFD9FF120066
:0A14E6001201000202000008D80401
:1014F0000A0000000102000109024300020100800D
:10150000FA09040000010202010005240010010490
:1015100024020205240600010524010001070582BA
:101520000308000209040100020A00000007050385
:101530000240000007058302400000040309043450
:10154000034D006900630072006F0063006800696A
:10155000007000200054006500630068006E006F9A
:10156000006C006F0067007900200049006E006386
:10157000002E002803550042005700200046006955
:101580000072006D0077006100720065002000436A
:10159000002000760030002E003100F814F8143BD3
:0715A000153F157315380813
:0815A8002A0EF66E080EF76E24
:1015B000000EF86E01010900F550056F0900F550A5
:1015C000066F03E1056701D03DD00900F550006FBB
:1015D0000900F550016F0900F550026F090009007C
:1015E000F550E96E0900F550EA6E0900090009009E
:1015F000F550036F0900F550046F09000900F6CF9C
:1016000007F1F7CF08F1F8CF09F100C1F6FF01C1EA
:10161000F7FF02C1F8FF0101035302E1045307E0A1
:101620000900F550EE6E0307F8E20407F9D707C189
:10163000F6FF08C1F7FF09C1F8FF01010507000E19
:06164000065BBFD712009B
:0A16460004D80FD8C8EC08F0FCD758
:101650000F0EC112140E6F6E0101126B0101136B9C
:101660000101146BB9EF08F0B8EC09F06FBE02D0BD
:08167000D4EC09F056EF05F07F
:08167800554257204669726DCE
:1016800077617265204320762742697473546F42F4
:0A1690007974657327312E300D00C8
:06169A0013EE00F023EE48
:1016A00000F0F86A019CD4EC0AF023EC0BF0FDD7B3
:0216B000120026
:0316B20001000034
:00000001FF
